:101AF2005343532D32313000013700000452533228
:101B0200333200000000000020380000004F7574DE
:101B12007075740000010D592038000000496E7084
:101B22007574000000010D790139000000426175F1
:101B32006400000000010D99000000000000000098
:081B420000000000000000009B
:081F7400017901030EFF1AFAC6
:10201500EF6006900D997403F0900D99E0FD7F0136
:08202500121C457F02021FF6A8
:0C17DC001511A811EFF6151115111511CB
:1017E800E5112403F8E67052900C19E05407A8118B
:1017F80008F6A81108087602A81108E6B4070CA391
:10180800E0A81108F6A81108087603A8110816A878
:1018180011E4F6A81108C9E8C9A811E6FFC3975052
:10182800170808E62F2419F582E4340CF583E0FF45
:10183800121E08A8110680DBD20FE5112403F8E672
:10184800FFB40102D210EFB4030A900D99E0FD7FB6
:0418580001121C4518
:07185C00E5112404F511223F
:101E4D00EF7039F536121CE48F35E535F4602AAFA5
:101E5D0036EF3395E0FE741B2FF582740D3EF5833E
:101E6D00E535F07A007B327D017F0112162F0536A4
:0E1E7D00C3E536648094A040CCAF36227F00CF
:011E8B002234
:101EC3008B358A368937120C38AB38AA39A93A12BE
:101ED3000C7EAB35AA36A937900001120C51AB38F2
:0D1EE300AA39A93A900001120C907F02224A
:1013AA00300F05C20F121FB8301053C210E4F50DEA
:1013BA00F53B7479253BF582E4340DF583E4F005B9
:1013CA003BE53BB420ECE4F53B7459253BF582E45C
:1013DA00340DF583E0FF601B121E08121FB87F0A46
:1013EA007E00121F497F00121F1D053BE53BC39477
:1013FA002040D612000E8F3F8E3E8D3D8C3C12004F
:10140A000EC3EF953FFFEE953EFEED953DFDEC9543
:10141A003CFCE47B2C7A01F9F8D3120D73402E12AE
:10142A001CE4EFF46022E50DC39420501BAE0D05B9
:10143A000D74792EF582E4340DF583EFF07A007B92
:10144A00327D017F0112162F7F00121F1D43870173
:01145A00226F
:0D205300245265763A2034393039202400BB
:10097000E47880F6122040C2B575840F75E104E476
:10098000F5E275E344F584F5B775840F758A83F550
:1009900097121FD7E4FF121FF643EF04E4F53DF56D
:1009A0003E7D01AF3E121EF0053EE53E7002053D64
:1009B000C39402E53D940040E8E4F520C20AC20871
:1009C000C20EC20DC20C7880F608F67854F618F6FE
:1009D0007859F6F53DF53E7419253EF582E4340C60
:1009E000F583E4F0053EE53E7002053DB400E8E520
:1009F0003DB401E3E4F53DF53E7419253EF582E48E
:100A0000340DF583E4F0053EE53E7002053D64409B
:100A1000453D70E5E4F584E5EF20E10CE5EF540891
:100A2000D394004003D38001C392037D08E4FF12F6
:100A30001C45E47858F67851F6AB0EAA0FA9107849
:100A400051E6FF75F010A4F58285F083120C51FE7B
:100A5000785826F6EE600578510680DDEFD39400D5
:100A60004030AB0EAA0FA91090000D120DDA120C37
:100A700038FF7455120C7E120C3864556002D20C8B
:100A800074AA120C7E120C3864AA6002D20CEF1207
:100A90000C7EE4F584E5EF5402D3940040047F011A
:100AA0008002E4FF12120D8F3CE53C20E036C209C3
:100AB00074FF785BF608F608F608F67E007F107D76
:100AC000007B007A007961120E307542FF75431A7F
:100AD0007544F27545007546107B007A0079611205
:100AE0001BF38002D20990205AE493FF3395E0FE75
:100AF000EF24D0FFEE34FFFE7C007D64120CB2AA1E
:100B000006AB07902059E493FF3395E0FEEF24D025
:100B1000FFEE34FFFE7C037DE8120CB2EF2BFBEE00
:100B20003AFA90205BE493FF3395E0FEEF24D0FF88
:100B3000EE34FFFE7C007D0A120CB2EF2BFFEE3A82
:100B4000FEA3E493FD3395E0FCED24D0FDEC34FFEF
:100B5000CD2F7860F6ED3E18F6E53C30E103020C4F
:100B60000FE4F53DF53EE53EC4F8540FC868FFE5D7
:100B70003DC454F048FEAB0EAA0FA9108F82F58336
:100B8000120C517003020C06E92FF9EA3EFA9000AC
:100B900004120C5120E264E4F53BE53BC3787996FE
:100BA0005059E53EC4F8540FC868FFE53DC454F001
:100BB00048AB0EAA0FA9108F82F583120C51FF7E4D
:100BC00000C006C0077D00E53EC4F8540FC868FFAA
:100BD000E53DC454F048FEE92FF9EA3EFA90000DD5
:100BE000120DDA7858E6853BF0A429F9EA35F0FAD7
:100BF000D007D006120E30053B809F053EE53E70C3
:100C000002053D020B667F01122015C20B8007E42E
:100C1000FF122015D20BE4F53DF53E7A007B967D60
:100C200003AF3E12162F053EE53E7002053DC3940C
:070C300002E53D940040E4E1
:010C3700229A
:050003007859E6FF2220
:03002300020EEEDC
:100EEE00C0E0C0F0C083C082C0D075D000C000C0CA
:100EFE0001C002C003C004C005C006C0073099403F
:100F0E00C2997854067954E77881667016F678544B
:010F1E00F6DC
:0E0F1F0075230A0075240300D524FCD523F5A4
:040F2D00C2B5801DAC
:0E0F31007523140075240300D524FCD523F588
:100F3F007854E62419F582E4340DF583E0F5992011
:100F4F009803020FEC209A08200A05C298020FE8B6
:100F5F00C29A7853E6062419F582E4340CF583E53A
:100F6F0099F0C298E6FFB40112900C19E0FE7003DD
:100F7F00F6806AEE54072402785AF6EFB4020D7821
:100F8F005AE6B40907900C1AE02403F67853E6FFEB
:100F9F00B40007E4B40103F68043EFC3785A9640D8
:100FAF003C7853E624FFFDE434FFFC7B017A0C7997
:100FBF00191217507853E62418F582E4340CF58390
:080FCF00E06F6004760080155C
:0E0FD7007523140075240300D524FCD523F5E2
:100FE5001200A678537600D007D006D005D004D0DD
:100FF50003D002D001D000D0D0D082D083D0F0D0A1
:02100500E032D7
:10002600900C1AE075F010A4AB0E2510F9E50F350B
:10003600F0FA90000D120DDA7859E6FF18E68FF007
:10004600A42527F582E435F0F583120C51FF7B00D9
:040056007A0079258E
:10005A008F358B368A378938E4F584EA494B601C38
:10006A00AB36AA37A938120C38FFE535FD7C0012E9
:0C007A002060AB36AA37A938EF120C7ECC
:0E00860075391400753A0300D53AFCD539F5EA
:0E0094008535997F01121F1D3099FDC29922FA
:101E8C00900D197478F07853E62418F582E4340C2C
:091E9C00F583E0900D1AF07F02BD
:091EA500E4F5847881EFF6D2B572
:0E1EAE007535140075360300D536FCD535F5B4
:071EBC00900D19E0F59922D9
:101D7900C9EFC9E964017028EDC39B40347879E65D
:101D8900FFEB2FFFE433FEEDC39FEE6480F8748010
:101D990098501ED20AC3ED9B7859F67855760122E0
:101DA900B90214ED6B700AD20A7859F678557602A1
:081DB90022C20AE47855F6226B
:101A9100C9EFC9BAFF15BBFF12ED6B7002EC6A709A
:101AA10049D20A7859F67855E9F622E96401702598
:101AB100C3ED9BEC9A401C7879E62BFFE43AFEC318
:101AC100ED9FEC9E500DD20AC3ED9B7859F67855E7
:101AD1007601228015B90218ED6B7002EC6A700A6A
:101AE100D20A7859F67855760222C20AE47855F678
:011AF10022D2
:1000A600900C19E0FF54F8F526E4F584EF120E0AD9
:1000B60000F30901000A011310011C11012D1201A0
:1000C6004419015A1A017F20018828020A29030DC2
:1000D60033034837037739039141039C4903A650FC
:1000E60003EE6102D77003E6980000041E900C1A16
:1000F600E0FD785CE6FB7F018027900C1AE0FCA30C
:10010600E0FD785BE6FA08E6FB7F01802BD20A78F1
:1001160055760302041E900C1AE0FD785EE6FB7F1E
:1001260002121D7902041E900C1AE0FCA3E0FD7871
:100136005DE6FA08E6FB7F02121A9102041E900C95
:100146001AE0FD785CE6FB7F01121D79200A0302A6
:10015600041E801A900C1AE0FCA3E0FD785BE6FA18
:1001660008E6FB7F01121A91200A0302041E900D75
:10017600197478F07F0102041BE4F58475EF100210
:10018600041EC2ACE4F525D2B5FB7A0079257F7F43
:1001960012005A7B007A0079257F1812005A7B00DC
:1001A6007A0079257F0512005A7851E612005378B5
:1001B6005BE6120053785CE6120053785DE61200A7
:1001C60053785EE6120053785FE61200537860E6D5
:1001D600120053E4F52774612527F8E6120053054B
:1001E60027E527C3941040EE7B007A007900AF25FF
:0301F60012005A9A
:0E01F90075330A0075340300D534FCD533F598
:100207000202C2900C1AE0FFC37851964003020223
:10021700C9EF75F010A42510F9E50F35F0850E30FC
:10022700F5318932C2ACE4F525D2B5FB7A007925E0
:100237007F7F12005A7B007A0079257F0D12005AC2
:10024700AB30AA31A932120C38120053AB30AA31A5
:10025700A932900001120050AB30AA31A9329000A8
:1002670002120050AB30AA31A9329000031200509D
:10027700AB30AA31A932900004120050E4F527AB45
:1002870030E5322405F9E43531FA7E00E92527F90E
:10029700EE3AFA120C381200530527E527C39408E3
:0D02A70040DD7B007A007900AF2512005A7F
:0E02B40075330A0075340300D534FCD533F5DC
:1002C200C2B5D2AC02041E900D197478F0E4A3F00A
:1002D2007F0202041B12202D7812120D91900D192B
:1002E200747CF07812E6A3F008E6A3F008E6A3F027
:1002F20008E6A3F07C007D057B017A0D79191217BF
:1003020050900D1EEFF07F0602041B900C1AE0FFC6
:10031200B4010FA3E0FDA3E0785BCDF608EDF60291
:1003220003E6EFB4020A900C1BE0785BF60203E6E8
:10033200900C1AE0B4030CA3E0FFA3E0785DCFF6C3
:1003420008EFF60203E6E4F527900C1AE0FFE52732
:10035200C39F501B741B2527F582E4340CF583E000
:10036200FF74612527F8EFF60527E527B410DAE4D4
:100372007870F6806F7A007B327D017859E6FF1241
:10038200162F900C1AE0FDE4FF121C4502041E9089
:100392000C1AE024FF920202041E900C1AE024FFC1
:1003A200920180787859E66005752902800B200D4C
:1003B200057529038003752901900D197479F0A33D
:1003C200E529F07C007D027B017A0D791912175024
:1003D200900D1BEFF07F03121EA5E5296401703C0E
:1003E200D20E8002D208788076F180307A007B3299
:1003F2007D017F0012162F900D197479F0900C1A5E
:10040200E0900D1AF07C007D027B017A0D791912C1
:100412001750900D1BEFF07F03121EA5E52664A076
:10042200600302062F900C19E064A1600302051E0E
:10043200A3E0C37851964003020513AB0EAA0FA99D
:1004420010E0FF75F010A4F58285F083120C51F5CF
:1004520029EF75F010A429F9EA35F0FA9000041298
:100462000C5130E237900C1AE0121E4D8F29900D7C
:1004720019747FF0A3E529F02402FDE433FC7B012B
:100482007A0D7919121750741B2529F582E4340D5F
:10049200F583EFF0E5292403FF02062C900C1AE005
:1004A200FF121E4DC2ACE4F525D2B5E529D3940660
:1004B200402B7B007A0079257F7F12005A7B007ADD
:1004C200007925AF2912005AE4F527E527C39529BB
:1004D2005007120026052780F205298018E52924F5
:1004E20078120053E4F527E527C395295007120037
:1004F20026052780F27B007A007900AF2512005A88
:0E05020075330A0075340300D534FCD533F58B
:1005100002061E900D197478F07F0102062C900CD3
:1005200019E064A2600302062F7851E6FFA3E0FE03
:10053000C39F4003020624A3E0FDC39F40030206BD
:1005400024EE9D4003020624900C1AE0F527E4F502
:100550002EF52F900C1BE0FFE527D39F5026AF27E9
:10056000121E4DAB0EAA0FA91075F010E527A4F5C9
:100570008285F083120C51252FF52FE4352EF52EB0
:10058000052780CFC2ACE4F525D2B5FB7A007925EA
:100590007F7F12005AC3E52F9480E52E940050020D
:1005A0008007E52E4480120053AF2F120054900CA8
:1005B0001AE0F527900C1BE0FFE527D39F5046E497
:1005C000F528AB0EAA0FA91075F010E527A4F58247
:1005D00085F083120C51FFE528C39F5024E5277551
:1005E000F010A429F9EA35F0FA90000D120DDA782E
:1005F00059E6FF18E68FF0A4252812004905288047
:10060000C1052780AF7B007A007900AF2512005A20
:0E06100075330A0075340300D534FCD533F57C
:10061E00C2B5D2AC800B900D197478F07F01121E0A
:10062E00A5E5266458704DFA7B327D017859E6FFB8
:10063E0012162F75380175390D753A1A7B017A0C21
:10064E00791A121EC38F29E5292478900D19F0EF1F
:10065E002401FDE433FC7B017A0D791912175074D5
:10066E001A2529F582E4340DF583EFF0E5292402ED
:10067E00FF121EA5E52664806009E52664886003E6
:10068E000208377855E6B4010F7A007B327D017887
:10069E0059E6FF12162F801AE4F527E527C378795D
:1006AE0096500F7A007B327D01AF2712162F052749
:1006BE0080E9900C19E05407F529B4070A75280152
:1006CE00A3E0F529A38006E4F528900C1AE0F52A9C
:1006DE001529E52AC37851964003020824AB0EAAC9
:1006EE000FA91075F010E52AA4F58285F083120C7F
:1006FE0051FFE529D39F40028F297855E6B40109B1
:10070E007859E6F52DF52C8009E4F52C7879E61468
:10071E00F52D7859A62C7859E6D3952D400302086D
:10072E0018E4F527E527C39529400302080DE52AAD
:10073E0075F010A4AB0E2510F9E50F35F0FA900008
:10074E0004120C5130E203020808900001120C5101
:10075E0064387041E529D394044011E528252724F7
:10076E001BF582E4340CF583E0FD80707853E6C30C
:10077E009527FFE49400FE74172FF582740C3EF556
:10078E0083E0FDE52A75F010A4AB0E2510F9E50FF8
:10079E0035F0FA8047AB0EAA0FA91075F010E52AB6
:1007AE00A4F58285F083120C51FF7853E6C39FFFA8
:1007BE00E49400FE7C00EF2527FFEC3EFEEF25289B
:1007CE00FFEC3EFE74182FF582740C3EF583E0FDAF
:1007DE00E52A75F010A429F9EA35F0FA90000D1209
:1007EE000DDA7859E6FF18E68FF0A4FFE5272FF50E
:1007FE0082E435F0F583ED120C900527020732AF37
:10080E002A1217DC7859060207247859A62CE526F9
:10081E00648870158010E52AB4FF0E900C1BE0F56D
:10082E0020E526B48803121E8CE52664A860030218
:10083E00096F7855E6B4010F7A007B327D01785945
:10084E00E6FF12162F801AE4F527E527C37879966E
:10085E00500F7A007B327D01AF2712162F052780AD
:10086E00E9900C1AE030E711547FFEA3E0FDEEF59F
:10087E002EEDF52F752803800C900C1AE0752E00C6
:10088E00F52F75280274192528F582E4340CF583AA
:10089E00E0FF741A2528F582E4340CF583E0F52B7D
:1008AE008F2AE52AD3952B400302096CE52AC378DB
:1008BE0051964003020967AB0EAA0FA91075F010EE
:1008CE00E52AA4F58285F083120C51F5297855E6B8
:1008DE00B401097859E6F52DF52C8009E4F52C784C
:1008EE0079E614F52D7859A62C7859E6D3952D5026
:1008FE005EE4F527E527C39529504AE52A75F010E1
:10090E00A4AB0E2510F9E50F35F0FA900004120C89
:10091E005120E22DE5282527241BF582E4340CF521
:10092E0083E0FD90000D120DDA7859E6FF18E68F80
:10093E00F0A4FFE5272FF582E435F0F583ED120CD8
:10094E0090052780AFAF2A1217DC785906809A7867
:10095E0059A62CE5292528F528052A0208B0121ECD
:01096E008CFC
:01096F002265
:107000007880E664F16003027630E4F540F541787B
:0470100081E6602095
:0E70140075460A0075470300D547FCD546F5C2
:107022000541E5417002054064107004E5406427A3
:1070320070DBC2AF7584015398FC75FFDE75FFAD3E
:10704200E4F53CF53BE4F58420982FE4F540F54166
:0E705200209823C3E5419488E540941350181C
:0E70600075460A0075470300D547FCD546F576
:10706E000541E54170DE054080DAB2B480CE8599E7
:10707E003BC298E53B641A6003027153F540F5413B
:0E708E00209823C3E5419488E54094135018E0
:0E709C0075460A0075470300D547FCD546F53A
:1070AA000541E54170DE054080DA30989085993CCB
:1070BA00C298E4F540F541209823C3E5419488E558
:0570CA00409413501872
:0E70CF0075460A0075470300D547FCD546F507
:1070DD000541E54170DE054080DA209803027047D6
:1070ED0085993CC298E4F540F541209823C3E541CC
:0870FD009488E540941350183B
:0E71050075460A0075470300D547FCD546F5D0
:107113000541E54170DE054080DA2098030270479F
:0971230085993CC298D2B5C299CD
:0E712C007546140075470300D547FCD546F59F
:06713A007599783099FD03
:0E71400075460A0075470300D547FCD546F595
:10714E00C2B5027622E53B645060030271E8F54059
:10715E00F541209823C3E5419488E54094135018D7
:0E716E0075460A0075470300D547FCD546F567
:10717C000541E54170DE054080DA20980302704736
:09718C0085993CC298D2B5C29964
:0E7195007546140075470300D547FCD546F536
:0871A3007599793099FDC2993C
:0E71AB007546140075470300D547FCD546F520
:0871B9007599013099FDC2999E
:0E71C1007546140075470300D547FCD546F50A
:0671CF00E4F5993099FD82
:0E71D50075460A0075470300D547FCD546F500
:0F71E300C2B5027622E53B64017041D2B5C29974
:0E71F2007546140075470300D547FCD546F5D9
:087200007599783099FDC299DF
:0E7208007546140075470300D547FCD546F5C2
:06721600E4F5993099FD3A
:0E721C0075460A0075470300D547FCD546F5B8
:10722A00C2B5027622E53B640260030272F5F540BC
:10723A00F541209823C3E5419488E54094135018FA
:0E724A0075460A0075470300D547FCD546F58A
:107258000541E54170DE054080DA20980302704759
:1072680085993CC298E4F53DE53C13B392B4E53CFE
:1072780025E0FEC3E49400EE9470502AE53C7F00BC
:1072880025E0FEC394E0501EE53C20E01FE4F584B1
:1072980043B701758F038E428F438F828E83F053DD
:1072A800B7F0F58F8003753DFFE4F584D2B5C29938
:0E72B8007546140075470300D547FCD546F512
:0872C6007599783099FDC29919
:0E72CE007546140075470300D547FCD546F5FC
:0672DC00853D993099FD8B
:0E72E20075460A0075470300D547FCD546F5F2
:1072F000C2B5027622E53B64036003027446F540A2
:10730000F541209823C3E5419488E5409413501833
:0E73100075460A0075470300D547FCD546F5C3
:10731E000541E54170DE054080DA20980302704792
:10732E0085993CC298E4F540F541209823C3E54188
:08733E009488E54094135018F7
:0E73460075460A0075470300D547FCD546F58D
:107354000541E54170DE054080DA2098030270475C
:1073640085993EC298E53C1392B4E53C25E0FEC302
:10737400E49400EE94704003027047E53C7D0025E0
:10738400E0FCC394E04003027047E4F58443B70192
:10739400758F01E53E75F020A42DFFE5F03CF54224
:1073A4008F43E4F584F53FE53FC394205049E4F569
:1073B40040F541209823C3E5419488E54094135057
:0173C40018B0
:0E73C50075460A0075470300D547FCD546F50E
:1073D3000541E54170DE054080DA209803027047DD
:1073E3000543E543AE427002054214F5828E83E500
:1073F30099F0C298053F80B0E4F58453B7F0F58F58
:06740300F584D2B5C29928
:0E7409007546140075470300D547FCD546F5BF
:087417007599783099FDC299C6
:0E741F007546140075470300D547FCD546F5A9
:06742D00E4F5993099FD21
:0E74330075460A0075470300D547FCD546F59F
:10744100C2B5027622E53B640460030274FAF5409A
:10745100F541209823C3E5419488E54094135018E1
:0E74610075460A0075470300D547FCD546F571
:10746F000541E54170DE054080DA20980302704740
:10747F0085993CC298E53C25E0F544754500E4F557
:10748F003DF540F5410545E545AE44700205441410
:10749F00F5828E83E493253DF53D0541E54170026C
:0E74AF0005407004E540640270DBD2B5C2995E
:0E74BD007546140075470300D547FCD546F50B
:0874CB007599783099FDC29912
:0E74D3007546140075470300D547FCD546F5F5
:0674E100853D993099FD84
:0E74E70075460A0075470300D547FCD546F5EB
:1074F500C2B5027622E53B64056003027617F540C6
:10750500F541209823C3E5419488E540941350182C
:0E75150075460A0075470300D547FCD546F5BC
:107523000541E54170DE054080DA2098030270478B
:1075330085993CC298E4F540F541209823C3E54181
:087543009488E54094135018F0
:0E754B0075460A0075470300D547FCD546F586
:107559000541E54170DE054080DA20980302704755
:0975690085993EC298D2B5C29981
:0E7572007546140075470300D547FCD546F555
:0875800075997F3099FDC29955
:0E7588007546140075470300D547FCD546F53F
:107596007599203099FDE53C25E0FCE53E75F02027
:1075A600A42400FFE5F03CF5448F45E4F53DF53FA6
:0275B600C29978
:0E75B8007546140075470300D547FCD546F50F
:1075C600854582854483E493F5993099FD0545E523
:1075D60045AE447002054414F5828E83E493253D3E
:0B75E600F53D053FE53FB420C7C2990A
:0E75F1007546140075470300D547FCD546F5D6
:0675FF00853D993099FD65
:0E76050075460A0075470300D547FCD546F5CB
:10761300C2B5800BE53BB40606E4F58475EF10E5CF
:0D7623003B640760030270477880F6D2AF29
:017630002237
:1018E2007F00121F1D121DC120090B7A007B327D61
:1018F200017F0012162F300C0B7A007B1E7D017FB8
:101902000012162F300817300D147A007B327D0139
:101912007859E6FF12162FC20812145BD209200B67
:101922000C300D09788076F112145BD20B300E0860
:10193200300D05C20E127000200D1212000EE47B53
:0E1942002C7A01F9F8C3120D735002D20D2257
:0B206C001209701218E21213AA80F88B
:10100700005EBCE2613FDD83C29C7E20A3FD1F41E1
:101017009DC3217FFCA2401E5F01E3BD3E6082DCD1
:10102700237D9FC1421CFEA0E1BF5D0380DE3C62C1
:10103700BEE0025CDF81633D7C22C09E1D43A1FFB1
:101047004618FAA427799BC584DA3866E5BB5907A1
:10105700DB856739BAE406581947A5FB7826C49A91
:10106700653BD987045AB8E6A7F91B45C6987A2481
:10107700F8A6441A99C7257B3A6486D85B05E7B971
:101087008CD2306EEDB3510F4E10F2AC2F7193CD61
:10109700114FADF3702ECC92D38D6F31B2EC0E5051
:1010A700AFF1134DCE90722C6D33D18F0C52B0EE41
:1010B700326C8ED0530DEFB1F0AE4C1291CF2D7331
:1010C700CA947628ABF517490856B4EA6937D58B21
:1010D7005709EBB536688AD495CB2977F4AA481611
:1010E700E9B7550B88D6346A2B7597C94A14F6A801
:1010F700742AC896154BA9F7B6E80A54D7896B35F1
:10110700000060B0CBD8E5F3F70096CBE5F3F7F92D
:0411170000000000D4
:101F7C00C192420C0D0009420C150009420C0F08CD
:091F8C0009420C17080901820A40
:1017500015111511A811ECF608EDF6151115111556
:1017600011A811C6EBC608C6EAC608C6E9C6E51147
:0417700024FCF5114F
:10177400F80808E4F6A811F608F6E5112407F9A814
:1017840011E6FE08E6FFC3099719E76480F8EE64E2
:1017940080985037E5112404F8CBE6CB08E6FA0824
:1017A400E6F98F828E83120C51A811080866FFE5B2
:1017B400112403F8EFF6E690100793A8110808F631
:1017C400A8110806E61870B20680AFA8110808E64A
:0117D400FF15
:0717D500E5112409F51122C2
:0B206000ED6F7816F6E690100793FF76
:01206B002252
:0300A300021863DD
:10186300C0E0C0F0C083C082C0D0E8C0E0EEC0E0FA
:10187300EFC0E0E59830E1055398FDD212E59830CA
:10188300E049900C16E02401FF900C15E03400FEB3
:10189300900C0DE06E7003A3E06F7002802A900C31
:1018A30015E475F001120CFA85F082F583E599F0E1
:1018B300900C15E064087004A3E06409700A900CAE
:1018C300157400F0A37409F05398FED0E0FFD0E044
:0F18D300FED0E0F8D0D0D082D083D0F0D0E03279
:101DC100900C0FE0FEA3E0FF900C17E06E7003A3F0
:101DD100E06F603230122FC212758401900C0FE453
:101DE10075F001120CFA85F082F583E0F599900CFB
:101DF1000FE0640C7004A3E06409700A900C0F7486
:071E010008F0A37409F022B0
:101BA100900C0DE0FEA3E0FF900C15E06E7003A316
:101BB100E06F6039900C0DE475F001120CFA85F0BC
:101BC10082F583E0781EF6900C0DE064087004A3A2
:101BD100E06409700A900C0D7400F0A37409F078A8
:101BE1001EE6FEB40D037F0A22CFEECF221218E2C9
:021BF10080AEC4
:021CE4001511D8
:101CE600900C0DE0FEA3E0FF900C15E06E7003A3D0
:101CF600E06F6031900C0DE475F001120CFA85F07E
:101D060082F583E0A811F6900C0DE064087004A338
:101D1600E06409700A900C0D7400F0A37409F0A831
:071D260011E6FF80027FFFC0
:031D2D000511227B
:0816C0008B088A09890A8D0BD1
:1016C80012000E787A120D91E4787EF6121CE4EF7F
:1016D800F46037EF640A6032BF0D13AB08AA09A99A
:1016E8000A787EE6FFF582758300E4020C90AB0869
:1016F800AA09A90A787EE606F582758300EF120C1E
:1017080090787EE6FF650B7001221218E212000E37
:10171800ECC0E0EDC0E0EEC0E0EFC0E0AF0CE4FCF0
:10172800FDFE787A120D84EF2BFBEE3AFAED39F9CB
:10173800EC38F8D0E0FFD0E0FED0E0FDD0E0FCD3FC
:07174800120D7350877F00B2
:01174F002277
:101E0800900C18E02401FD900C17E03400FC900CB5
:101E18000FE06C7003A3E06D700122900C17E4755D
:101E2800F001120CFA85F082F583EFF0900C17E0C0
:101E3800640C7004A3E06409700A900C177408F02D
:051E4800A37409F02263
:101FB800900C0FE0FEA3E0FF900C17E06E7003A3F7
:0F1FC800E06F600A7F00121F1D121DC180E22210
:101D30007E007F09900C15EEF0A3EFF0900C0DEEF5
:101D4000F0A3EFF07E087F09900C17EEF0A3EFF000
:101D5000900C0FEEF0A3EFF07E087F007D007B017A
:101D60007A007909120E307E047F007D007B017AB3
:091D7000087909120E30D212228A
:101C4500EF7025F5847598D0F584759115F5847533
:101C5500C90875CBFFED90110693F5CA75C804E464
:101C6500F584D2ACC2BC8026758401759850E4F524
:101C750084E589540F4420F589758E02ED90111085
:101C850093F58DD28E43E74053F7BF121D30D2AF87
:011C9500222C
:1019BE00900C09120DA900000000900C11120DA937
:1019CE00000000009000007464F0E47817F67817B9
:1019DE00E6FFC394025043EF25E025E02401F58293
:1019EE00E43400F583E4F0EF25E025E02402F582EF
:1019FE00E43400F583E4F0EF25E025E02403F582DE
:101A0E00E43400F583E4F0EF25E025E02404F582CC
:0A1A1E00E43400F583E4F00680B420
:011A2800229B
:101FD700D2AFD2A9C2BBE4F584E589540F4401F519
:0F1FE70089758E02758CECE4F58AD28C0219BED6
:02111B001511AC
:10111D00A811E4F6A811E6FFC39402400302120AD7
:10112D00EF25E025E02404F582E43400F583E0FFAB
:10113D00D3940050030211DFE625E025E02402F5EB
:10114D0082E43400F583E060030211DFEF30E01933
:10115D00E6FF25E025E02404F582E43400F583E084
:10116D00D3940140047D0080067D01A811E6FF1295
:10117D001950A811E6FF25E025E02404F582E4349A
:10118D0000F583E0B401057D01121950A811E6FFA9
:10119D0025E025E02404F582E43400F583E014F025
:1011AD00EF25E025E02404F582E43400F583E060CA
:1011BD0021E6FF25E025E02403F582E43400F583E4
:1011CD00E0FEEF25E025E02402F582E43400F5830E
:1011DD00EEF0A811E6FF25E025E02402F582E434C7
:1011ED0000F583E06011EF25E025E02402F582E4AF
:0D11FD003400F583E014F0A8110602112162
:03120A00051122A9
:03000B000214FEDE
:1014FE00C0E0C0F0C083C082C0D0E8C0E0E9C0E068
:10150E00EAC0E0EBC0E0ECC0E0EDC0E0EEC0E0EF22
:10151E00C0E0758CEC900C09E0FCA3E0FDA3E0FEAE
:10152E00A3E02401FFE43EFEE43DFDE43CFC900C10
:10153E0009120D9D900000E014F0E07025900C1142
:10154E00E0FCA3E0FDA3E0FEA3E02401FFE43EFEE9
:10155E00E43DFDE43CFC900C11120D9D90000074D6
:10156E0064F012111B121F96D0E0FFD0E0FED0E007
:10157E00FDD0E0FCD0E0FBD0E0FAD0E0F9D0E0F80E
:0B158E00D0D0D082D083D0F0D0E0326B
:101EF0001511A811EDF61511A811EFF6A811E6FFBE
:101F0000C39402501308E6FEEF25E025E02401F516
:0D1F100082E43400F583EEF0051105112286
:10162F0015111511A811EAF608EBF61511A811ED11
:10163F00F61511A811EFF6A811E6FFC39402506A30
:10164F00EF25E025E02404F582E43400F583E07013
:10165F0059E6FB25E025E02402F582E43400F5830A
:10166F00E0704708E625E004FFA811E6FA25E0251B
:10167F00E02404F582E43400F583EFF00808E6FE79
:10168F0008E6FF7C007D0A120CC4EA25E025E02461
:10169F0003F582E43400F583EFF0EB25E025E02439
:1016AF0002F582E43400F583E4F0E5112404F5112A
:0116BF002208
:0E1950001511A811EDF61511A811EFF61511DD
:10195E00A81108E6FFC394025024EF25E025E024E9
:10196E0001F582E43400F583E06013A8110808E65F
:10197E0070047F0180027F00A8110808EFF6A811FD
:10198E00A68475840FA81108E6FF700BA81108082D
:10199E00E624FF92B4800DEFB40109A8110808E601
:0919AE0024FF92B3A811E6F584B0
:0719B70005110511051122C5
:10000E00C2AF900C09E0FCA3E0FDA3E0FEA3E0FF6D
:02001E00D2AF5F
:0100200022BD
:10202D00C2AF900C11E0FCA3E0FDA3E0FEA3E0FF26
:02203D00D2AF20
:01203F00227E
:101F1D001511A811EFF6A811E670057883F608F6ED
:101F2D003011167882E675F064A4FFC37884E69FBD
:0C1F3D0018E695F0500375FFA505112271
:101FF600D211E47883F608F6EF78826003F6800261
:0F200600760A75FF0775FFA5E4F58475EF0422D0
:10204000C211E47883F608F6788276FF75FFDE75B4
:03205000FFAD22BF
:101F9600788406E6187001063011167882E675F028
:101FA60064A4FFC37884E69F18E695F0500375FF96
:021FB600A52262
:041F49008E408F41F6
:101F4D00E4F542F543C3E5439541E542954050160E
:101F5D007FE87E03121B4A7F01121F1D0543E543D7
:061F6D0070E3054280DF75
:011F7300224B
:041B4A008E448F45F1
:101B4E00D3E54594FAE5449400500FEFD39400404A
:101B5E0041007E0300DEFD1F80F18544468545472A
:101B6E00D3E54794FAE546940040157FFA7E0012BD
:101B7E001B4A74062547F54774FF3546F54680E047
:101B8E00D3E5459400E54494004007AF47AE4612B6
:021B9E001B4AE0
:011BA0002222
:101A2900754B00754C00754D457B007A0079437DF7
:011A390002AA
:081A3A008B478A4889498D4A57
:101A42007F01121F1DAB4BAA4CA94D120D10240091
:101A5200FFE5F034E0FE85474E85484F854950E466
:101A6200FDEDC3954A501BEF2DF582E43EF583E46C
:101A720093AB4EAA4FA9508D82758300120C900D24
:0F1A820080DFAB4BAA4CA94DE4854AF0020D3B27
:1012F500753D12753E3475450075460075473F7B53
:07130500007A00793D7D0232
:08130C008B418A4289438D44A4
:101314007880E664F160030213A9122040C2AFE4AE
:10132400F58443B701758F01AB45AA46A947120D51
:10133400102400FFE5F034E07817F608EFF6AA422F
:10134400A943781BA64108C6EAC608C6E9C6E478DC
:1013540019F67819E6C395445032781BCBE6CB08CE
:101364000806E618CAE6CA70010614F9120C3878A1
:101374001AF6E6FF78170806E618CCE6CC700106E4
:1013840014F5828C83EFF078190680C6E4F58F5348
:10139400B7F0AB45AA46A9478544F0120D3BD2AF3E
:0513A400E4FF121FF63A
:0113A9002221
:101C96007880E664F17046C2AF122040E4F58443D2
:101CA600B701758F03781876E008F67817F6781876
:101CB600E6FE08E6F5828E83E4F07F01121F1D78AA
:101CC60019E426F618740236F61806E6C394084098
:0D1CD600DDE4F58F53B7F0D2AFFF121FF61B
:011CE30022DE
:10145B00121C96E4F53FF540F54575460075473F80
:10146B00FB7A00795B7D1612130C1212F5E4F53C36
:10147B00E53CC37879965073E4F53BAB0EAA0FA904
:10148B001075F010E53BA4F58285F083120C5160CA
:10149B0056E53B75F010A429F9EA35F0FA90000DEA
:1014AB00120DDA7858E6853CF0A429F9EA35F0FA02
:1014BB00EBC0E0EAC0E0E9C0E0AB0EAA0FA91075E3
:1014CB00F010E53BA4F58285F083120C51FD7545B8
:1014DB000075460075473FD0E0F9D0E0FAD0E0FB4D
:1014EB0012130C053B8094053C80851212F5E478B1
:0214FB0080F679
:0114FD0022CC
:02120D008F3F11
:10120F00E4F545F546F542F54B754C00754D45FB3C
:10121F007A00795B7D16121A3A121A29E544643462
:10122F007004E54364127003434201E4F541E54164
:10123F00C378799640030212E0E4F540AB0EAA0F93
:10124F00A91075F010E540A4F58285F083120C51BA
:10125F00607AE53F6054E54075F010A429F9EA354E
:10126F00F0FA90000D120DDA7858E68541F0A429B6
:10127F00F9EA35F0FAEBC0E0EAC0E0E9C0E0AB0E06
:10128F00AA0FA91075F010E540A4F58285F083121E
:10129F000C51FD754B00754C00754D45D0E0F9D0E4
:1012AF00E0FAD0E0FB121A3A801DAB0EAA0FA9107C
:1012BF0075F010E540A4F58285F083120C51254698
:1012CF00F546E43545F545054002124B054102123E
:1012DF003D121A29E54464347004E5436412700327
:0512EF00434202AF4282
:0112F40022D7
:030000000215994D
:1015990075840075EF027864D8FE787FE4F6D8FD8B
:0615A9007581840215EAC1
:1015AF0002206CE493A3F8E493A34003F68001F2C6
:1015BF0008DFF48029E493A3F85407240CC8C3333D
:1015CF00C4540F4420C8834004F456800146F6DF0C
:1015DF00E4800B0102040810204080901F74E47E09
:1015EF00019360BCA3FF543F30E509541FFEE49301
:1015FF00A360010ECF54C025E060A840B8E493A3C8
:10160F00FAE493A3F8E493A3C8C582C8CAC583CAF2
:10161F00F0A3C8C582C8CAC583CADFE9DEE780BEAA
:011F9500004B
:100C3800BB010689828A83E0225002E722BBFE02BA
:090C4800E32289828A83E49322ED
:100C5100BB010CE58229F582E5833AF583E0225058
:100C610006E92582F8E622BBFE06E92582F8E222A2
:0D0C7100E58229F582E5833AF583E49322BC
:100C7E00BB010689828A83F0225002F722BBFE0155
:020C8E00F3224F
:100C9000F8BB010DE58229F582E5833AF583E8F09A
:100CA000225006E92582C8F622BBFE05E92582C846
:020CB000F2222E
:100CB200EF8DF0A4A8F0CF8CF0A428CE8DF0A42E56
:020CC200FE2210
:100CC400C2D5EC30E709B2D5E4C39DFDE49CFCEE4B
:100CD40030E715B2D5E4C39FFFE49EFE120E5CC359
:100CE400E49DFDE49CFC8003120E5C30D507C3E454
:060CF4009FFFE49EFE22BA
:100CFA00A3F8E0C5F025F0F0E582158270021583AD
:060D0A00E0C838F0E82209
:100D1000BB010A89828A83E0F5F0A3E022500687AE
:100D2000F009E71922BBFE07E3F5F009E319228970
:0B0D3000828A83E493F5F074019322A3
:100D3B00BB010789828A83020EB1500B09C5F027CC
:100D4B00F7C5F01937F722BBFE0D09F8E325F0F3D1
:100D5B00C5F019E338F322F889828A83740193254D
:080D6B00F0C5F0F8E493382212
:100D7300EB9FF5F0EA9E42F0E99D42F0E89C45F0D6
:010D8300224D
:0D0D8400E6FB08E6F908E6FA08E6CBF822DF
:0C0D9100ECF608EDF608EEF608EFF6228E
:0C0D9D00ECF0A3EDF0A3EEF0A3EFF022C9
:100DA900A8828583F0D083D082120DC0120DC012A3
:100DB9000DC0120DC0E473E493A3C583C5F0C583C8
:100DC900C8C582C8F0A3C583C5F0C583C8C582C894
:010DD90022F7
:100DDA00BB010DE58229F582E5833AF583020ED03F
:100DEA005007E92582F8020EC7BBFE07E92582F8FB
:100DFA00020ED9E58229F582E5833AF583020EE2ED
:100E0A00D083D082F8E4937012740193700DA3A377
:100E1A0093F8740193F5828883E47374029368608B
:060E2A00EFA3A3A380DF8B
:101BF3008B3F8A408941E4F547F548E5461546AEF3
:101C030045700215454E6033AB42AA43A944120CFA
:101C130038FFAB3FAA40A9410548E548AC477002ED
:101C2300054714F5828C83EF120C90EF60CD74019D
:101C33002544F544E43543F54380C0AB3FAA40A9AE
:021C430041223C
:100E3000EF4E6012EF60010EEDBB010B89828A83D9
:100E4000F0A3DFFCDEFA2289F05007F709DFFCA9E6
:0C0E5000F022BBFEFCF309DFFCA9F0223D
:100E5C00BC000BBE0029EF8DF084FFADF022E4CC7A
:100E6C00F875F008EF2FFFEE33FEEC33FCEE9DEC43
:100E7C00984005FCEE9DFE0FD5F0E9E4CEFD22ED89
:100E8C00F8F5F0EE8420D21CFEADF075F008EF2FD3
:100E9C00FFED33FD4007985006D5F0F222C398FDC4
:050EAC000FD5F0EA2261
:100EB100C5F0F8A3E028F0C5F0F8E58215827002CC
:060EC1001583E038F02269
:090EC700E6FB08E6FA08E6F92250
:090ED000E0FBA3E0FAA3E0F92223
:090ED900E2FB08E2FA08E2F9224A
:0C0EE200E493FB740193FA740293F9226C
:00000001FF
